:1000000000308A004E2900002908AB008316051233
:100010008312051283160511831205110130AA00FF
:100020002A08083C031C30282B3084000008803943
:10003000003A031D20288316851183128511242878
:1000400083168511831285150310AB0D83160512D7
:10005000831205168316051283120512AA0A1028A8
:1000600083160511831205150034A401A5011F157F
:100070001F1938281E08A701A6000310A60DA70DFA
:1000800003178E010313240803178D0083168C13A6
:100090000C1483120C080313A800A9000420A40A5E
:1000A00022082402031C5528A4012608270403194A
:1000B0005E2826080319A703A603552883160517EB
:1000C0008312051B6428652837287429A601260891
:1000D000023C031C7C282508A90004204230F700BC
:1000E000F70B70280000A90104204230F700F70B3D
:1000F00077280000A60A67280034A4012408803C61
:10010000031CA12803178E010313240803178D0075
:100110008C0183168C130C15831203130B08F70044
:100120008B138316031755308D00AA308D008C1465
:100130008C1898280C117708831203138B04A40AD7
:100140007E28A401FF30A5006620FF3083168600BC
:1001500083120608FF3AA3002308A900042083168F
:1001600085168312851A262903178E010313240886
:1001700003178D000313230803178C0083168C13B9
:100180000C15831203130B08F7008B138316031748
:1001900055308D00AA308D008C148C18CD280C1190
:1001A0007708831203138B04A308031DDB28FF3099
:1001B000A5006620DE282308A50066201030F70081
:1001C000F70BE0280000831685168312851AEE28A7
:1001D0001830F700F70BEA2800000000A40A2408F2
:1001E0007D3C03182529831605178312051B062954
:1001F000FF30A90004202130F700F70BFD28A901EA
:1002000004202130F700F70B0329F32803178E0190
:100210007F308D007E308C0083168C130C1583127A
:1002200003130B08F7008B138316031755308D004B
:10023000AA308D008C148C181B290C11770883129E
:1002400003138B047E30F8004D294C2983160517C3
:100250008312051F4C2903178E017F308D00031375
:10026000240803178C0083168C130C1583120313B8
:100270000B08F7008B138316031755308D00AA3037
:100280008D008C148C1842290C11770883120313EB
:100290008B042408F8004D29A528762984011F30F5
:1002A0008305063083169F0081139F0183121F0868
:1002B0003839C1389F000830F8001F08C739780462
:1002C0009F0003178E017F308D0083168C130C1452
:1002D00083120C080313A100831605178312051F50
:1002E00075292108A200352878297D287808A100E1
:0402F0006C29630012
:02400E00101F81
:00000001FF
